:100000000C9441020C945E020C945E020C945E020D
:100010000C945E020C945E020C945E020C94FE0A38
:100020000C945E020C945E020C94FD0C0C945E0227
:100030000C945E020C94B7080C94E5080C945E02D4
:100040000C945E020C945E020C945E020C945E02B0
:100050000C945E0276322E332052656C65617365B6
:100060000A00496E697469616C697A65643A2000B6
:1000700053656C662D54657374204572726F723AC5
:1000800020306200203D3E204E6F20616E73776508
:10009000722066726F6D20417564696F210A0020BD
:1000A0003D3E204E6F20616E737765722066726FE1
:1000B0006D204D656D6F7279210A00203D3E204311
:1000C000616E277420777269746520746F204D65A6
:1000D0006D6F7279210A00286429656C6574652C3E
:1000E00020286729657420616E696D732C20287340
:1000F00029657420616E696D732C202876296572DC
:1001000073696F6E0A00287429696D652C20286157
:10011000297564696F2C202863296F756E742C20F3
:10012000287829437573746F6D20636F756E740A38
:100130000028792953657420666978656420616EAA
:10014000696D6174696F6E20636F756E740A005318
:100150002865296C6620546573742C20286D296FDE
:1001600064650A00506C61792053286E29616B65C3
:100170000A00416C6C204C454473204F66662F4F3B
:100180006E2028302F31290A002832293A20546560
:10019000737420416E696D2E20310A002833293A8C
:1001A00020416C6C2053757266616365204C454438
:1001B00073206F6E0A0053797374656D2054696DF6
:1001C000653A2000204672616D65732073746F720A
:1001D00065640A0053656E64206120627974652E3F
:1001E0002E2E2000207772697474656E210A0041FA
:1001F0006E696D6174696F6E20636F756E74206EC9
:100200006F772038373035210A0053656C662D54DE
:100210006573743A203062004B696C6C65642041F0
:100220006E696D6174696F6E20436F756E7465726F
:10023000210A00436F756C64206E6F7420616363E4
:1002400065737320646576696365210A004175648E
:10025000696F20446174613A0A00436F6E74726F73
:100260006C733A2057204120532044205120452CC4
:10027000207820746F20717569740A0052616E20B5
:100280006F7574206F662048656170210A00416EA9
:10029000696D6174696F6E2061626F72746564214B
:1002A0000A002869296E7465727275707420636F14
:1002B000756E742C20287229616E646F6D2C202855
:1002C000712972657365740A0020496E74657272D3
:1002D0007570747320616674657220313030306DD2
:1002E0007365630A00204672616D657320706572E4
:1002F000205365636F6E640A004D656D6F727920DF
:1003000064656C65746564210A00526573657420C8
:10031000696E203530306D732E20427965210A00D8
:100320005761746368646F672052657365742064F5
:10033000657465637465642E0A0042726F776E2D72
:100340004F757420526573657420646574656374B9
:1003500065642E0A004E6F205265736574207265C5
:1003600061736F6E2064657465637465642E0A0042
:1003700045787465726E616C205265736574206493
:10038000657465637465642E0A004A5441472052BF
:10039000657365742064657465637465642E0A0012
:1003A000506F7765722D4F6E2052657365742064AF
:1003B000657465637465642E0A0059617921204172
:1003C0006E6F74686572206D696E757465207061FA
:1003D00073736564203A290A00417564696F204D82
:1003E0006F6465210A0043756265204D6F64652165
:1003F0000A0043756265206D6F646520656E7465E3
:10040000726564210A00417564696F206D6F6465CF
:1004100020656E7465726564210A00540070006284
:100420000084009F00BB00D700060131014F01642A
:1004300001720189019C01B601C401D401E401EFFC
:10044000010A02180233024D025A027C028E02A2F5
:1004500002C902E502F9020A0320033A03550370B8
:10046000038A03A003BA03D903E603F20306045385
:100470007472696E67206E6F7420666F756E64218A
:100480000A0011241FBECFE5D8E0DEBFCDBF11E0CA
:10049000A0E6B0E0ECEDFFE102C005900D92A237BE
:1004A000B107D9F712E0A2E7B1E001C01D92A6356D
:1004B000B107E1F70E9476070C94EC0F0C94000052
:1004C000B0990AC080917301882321F481E0809360
:1004D000730102C0109273018091730108957F929D
:1004E0008F929F92AF92BF92CF92DF92EF92FF9244
:1004F0000F931F93CF93DF930E948C0D7C016FEFBE
:1005000070E00E94CC0E892B39F4C7016FEF70E0C8
:100510000E94CC0E762E07C0C7016FEF70E00E94DC
:10052000CC0E762E739482E40E94BF09872D0E9420
:10053000BF090E946A0990E08234910509F061C008
:10054000AA24BB244BC08FEFE816F10421F018F069
:1005500088248A9401C08E2C882D0E94BF090E9495
:100560006A0990E08234910509F04BC06501992435
:100570002DC0C6010E94FF0D8C01FC01E05CFF4F05
:1005800080810E94BF090E946A0990E0823491052F
:10059000A9F4C0E0D0E0F801EC0FFD1F80810E94BB
:1005A000BF092196C034D105B1F70E946A0990E0D5
:1005B0000894C11CD11C8234910521F0C8010E940D
:1005C0008D0F1FC0C8010E948D0F9394981488F25C
:1005D000E818F1088FEF90E0A80EB91E8A2D8195DA
:1005E000871508F4B0CF82E40E94BF0982E40E941C
:1005F000BF0982E40E94BF0982E40E94BF090E94F1
:100600006A09DF91CF911F910F91FF90EF90DF90DA
:10061000CF90BF90AF909F908F907F9008952F9232
:100620003F924F925F926F927F928F929F92AF9282
:10063000BF92CF92DF92EF92FF920F931F93DF93BF
:10064000CF93CDB7DEB727970FB6F894DEBF0FBEB6
:10065000CDBF81E490E00E94E00E7C010E946C0D11
:10066000422E332E242E752E662E572E982E892E2E
:1006700082E40E94BF096CC00E946C0D022F041915
:10068000F1E0201708F0F0E0232F2319E1E0321702
:1006900008F0E0E0A22FAF1B31E02A1708F030E0AD
:1006A000E32B242F2219F1E0421708F0F0E0B22FDB
:1006B000BE1B31E02B1708F030E0F32B252F271954
:1006C00041E0521708F040E0E22FEF1B31E02E1717
:1006D00008F030E0432B262F261951E0621708F06E
:1006E00050E0622F641B31E0261708F030E0532BF6
:1006F000272F251941E0721708F040E0322F351BF3
:10070000532F31E0251708F030E0432B282F29190B
:1007100031E0821708F030E0822F841B482F81E0FF
:10072000241708F080E0382B9819931789F4442394
:1007300079F4552369F4662359F4EE2349F4BB2375
:1007400039F4A83228F4A73211F4013108F4A8953D
:100750000E945B09882309F48FCF0E946A098A836B
:1007600082E40E94BF091B82AA24BB24F701E05C3B
:10077000FF4FFD83EC8388C10E946C0D022F04198A
:10078000F1E0201708F0F0E0232F2319E1E0321701
:1007900008F0E0E0A22FAF1B31E02A1708F030E0AC
:1007A000E32B242F2219F1E0421708F0F0E0B22FDA
:1007B000BE1B31E02B1708F030E0F32B252F271953
:1007C00041E0521708F040E0E22FEF1B31E02E1716
:1007D00008F030E0432B262F261951E0621708F06D
:1007E00050E0622F641B31E0261708F030E0532BF5
:1007F000272F251941E0721708F040E0F22FF51B72
:100800005F2F31E02F1708F030E0432B282F2919F4
:1008100031E0821708F030E0822F841B482F81E0FE
:10082000241708F080E0382B9819931789F4442393
:1008300079F4552369F4662359F4EE2349F4BB2374
:1008400039F4A83228F4A73211F4013108F4A8953C
:100850000E945B09882309F48FCF0E946A0989836B
:1008600082E40E94BF09650104C10E946C0D022F41
:100870000419F1E0201708F0F0E0232F2319E1E03C
:10088000321708F0E0E0A22FAF1B31E02A1708F082
:1008900030E0E32B242F2219F1E0421708F0F0E0BA
:1008A000B22FBE1B31E02B1708F030E0F32B252FC1
:1008B000271941E0521708F040E0E22FEF1B31E02A
:1008C0002E1708F030E0432B262F261951E062172F
:1008D00008F050E0622F641B31E0261708F030E08A
:1008E000532B272F251941E0721708F040E0F22F13
:1008F000F51B5F2F31E02F1708F030E0432B282F36
:10090000291931E0821708F030E0822F841B482F2C
:1009100081E0241708F080E0382B9819931789F4A8
:10092000442379F4552369F4662359F4EE2349F4FA
:10093000BB2339F4A83228F4A73211F4013108F4AA
:10094000A8950E945B09882309F48FCF0E946A0949
:10095000EC81FD81808382E40E94BF09FF82EE82E8
:100960006CC00E946C0D022F0419F1E0201708F0F2
:10097000F0E0232F2319E1E0321708F0E0E0A22F86
:10098000AF1B31E02A1708F030E0E32B242F2219A7
:10099000F1E0421708F0F0E0B22FBE1B31E02B1758
:1009A00008F030E0F32B252F271941E0521708F00B
:1009B00040E0E22FEF1B31E02E1708F030E0432B30
:1009C000262F261951E0621708F050E0622F641BB1
:1009D00031E0261708F030E0532B272F251941E08E
:1009E000721708F040E0F22FF51B5F2F31E02F1750
:1009F00008F030E0432B282F291931E0821708F046
:100A000030E0822F841B482F81E0241708F080E01B
:100A1000382B9819931789F4442379F4552369F4F2
:100A2000662359F4EE2349F4BB2339F4A83228F4A1
:100A3000A73211F4013108F4A8950E945B098823BC
:100A400009F48FCF0E946A09EE81FF818193FF83B1
:100A5000EE832C813D81E217F30779F782E40E944F
:100A6000BF0986010F5F1F4FC601B7010E94E80D45
:100A700068018C2D8A193981831708F462CFA30E7F
:100A8000B11C8B818F5F8B839B81EA819E1708F459
:100A9000DFCEC7010E948D0F6CC00E946C0D022F2B
:100AA0000419F1E0201708F0F0E0232F2319E1E00A
:100AB000321708F0E0E0A22FAF1B31E02A1708F050
:100AC00030E0E32B242F2219F1E0421708F0F0E088
:100AD000B22FBE1B31E02B1708F030E0F32B252F8F
:100AE000271941E0521708F040E0E22FEF1B31E0F8
:100AF0002E1708F030E0432B262F261951E06217FD
:100B000008F050E0622F641B31E0261708F030E057
:100B1000532B272F251941E0721708F040E0F22FE0
:100B2000F51B5F2F31E02F1708F030E0432B282F03
:100B3000291931E0821708F030E0822F841B482FFA
:100B400081E0241708F080E0382B9819931789F476
:100B5000442379F4552369F4662359F4EE2349F4C8
:100B6000BB2339F4A83228F4A73211F4013108F478
:100B7000A8950E945B09882309F48FCF0E946A0917
:100B80006CC00E946C0D022F0419F1E0201708F0D0
:100B9000F0E0232F2319E1E0321708F0E0E0A22F64
:100BA000AF1B31E02A1708F030E0E32B242F221985
:100BB000F1E0421708F0F0E0B22FBE1B31E02B1736
:100BC00008F030E0F32B252F271941E0521708F0E9
:100BD00040E0E22FEF1B31E02E1708F030E0432B0E
:100BE000262F261951E0621708F050E0622F641B8F
:100BF00031E0261708F030E0532B272F251941E06C
:100C0000721708F040E0F22FF51B5F2F31E02F172D
:100C100008F030E0432B282F291931E0821708F023
:100C200030E0822F841B482F81E0241708F080E0F9
:100C3000382B9819931789F4442379F4552369F4D0
:100C4000662359F4EE2349F4BB2339F4A83228F47F
:100C5000A73211F4013108F4A8950E945B0988239A
:100C600009F48FCF0E946A096CC00E946C0D022F9C
:100C70000419F1E0201708F0F0E0232F2319E1E038
:100C8000321708F0E0E0A22FAF1B31E02A1708F07E
:100C900030E0E32B242F2219F1E0421708F0F0E0B6
:100CA000B22FBE1B31E02B1708F030E0F32B252FBD
:100CB000271941E0521708F040E0E22FEF1B31E026
:100CC0002E1708F030E0432B262F261951E062172B
:100CD00008F050E0622F641B31E0261708F030E086
:100CE000532B272F251941E0721708F040E0F22F0F
:100CF000F51B5F2F31E02F1708F030E0432B282F32
:100D0000291931E0821708F030E0822F841B482F28
:100D100081E0241708F080E0382B9819931789F4A4
:100D2000442379F4552369F4662359F4EE2349F4F6
:100D3000BB2339F4A83228F4A73211F4013108F4A6
:100D4000A8950E945B09882309F48FCF0E946A0945
:100D50006CC00E946C0D022F0419F1E0201708F0FE
:100D6000F0E0232F2319E1E0321708F0E0E0A22F92
:100D7000AF1B31E02A1708F030E0E32B242F2219B3
:100D8000F1E0421708F0F0E0B22FBE1B31E02B1764
:100D900008F030E0F32B252F271941E0521708F017
:100DA00040E0E22FEF1B31E02E1708F030E0432B3C
:100DB000262F261951E0621708F050E0622F641BBD
:100DC00031E0261708F030E0532B272F251941E09A
:100DD000721708F040E0F22FF51B5F2F31E02F175C
:100DE00008F030E0432B282F291931E0821708F052
:100DF00030E0822F841B482F81E0241708F080E028
:100E0000382B9819931789F4442379F4552369F4FE
:100E1000662359F4EE2349F4BB2339F4A83228F4AD
:100E2000A73211F4013108F4A8950E945B098823C8
:100E300009F48FCF0E946A0982E40E94BF09C501AC
:100E40000E94B70D81E08093600027960FB6F8945A
:100E5000DEBF0FBECDBFCF91DF911F910F91FF90ED
:100E6000EF90DF90CF90BF90AF909F908F907F904A
:100E70006F905F904F903F902F900895863561F16D
:100E8000873580F4873411F1883438F48234E1F006
:100E90008434C1F08F3331F513C0883489F0833541
:100EA00009F517C0883661F0893628F4843651F088
:100EB0008736C1F40BC0833761F0863799F40CC0D4
:100EC00086E00BC00E94C90D82E40DC00E946F0233
:100ED00008950E940F03089580E00E94110E0E9461
:100EE000FC09089583E20E94BF0908954F925F9222
:100EF0006F927F928F929F92AF92BF92CF92DF922A
:100F0000EF92FF920F931F93CF93DF9384B7809359
:100F10008E0114BE98E10FB6F89491BD11BC0FBEBE
:100F20008FEF8ABB8CEF81BB97BB84BB87B3866096
:100F300087BBB8980E94830A89E190E068E040E0AE
:100F400021E00E9427090E94780B0E94F40C7894FB
:100F50002EE088E190E00FB6F894A89581BD0FBE11
:100F600021BD81E690E00E94290A0E946002482E7D
:100F70000E946C0D522E632E742E852E962EA72E57
:100F8000B82EC92E0E948C0DEC01EE24DD24FF2426
:100F900080917201882309F4A895442069F00E9489
:100FA0007F0A882309F463C00E94D50C009709F4D6
:100FB0005EC00E94730E5BC080916000882331F098
:100FC0000E948C0DEC0110926000EE24209709F134
:100FD0000E947F0AD81608F04AC02E2D30E0CE01BC
:100FE00001972817390710F0EE2401C0E3948E2DE5
:100FF00090E00E94FF0D8C01005C1F4FF801D08033
:1010000000541040C8010E94290AC8010E948D0F97
:101010002EC08091740182FD2AC081FF0FC00E9402
:10102000AE0EF81638F41F2D1F5F8F2D0E94B00EE4
:10103000F12E1DC0809174018D7F16C00E947F0A21
:101040008033A8F0EF2DF0E0EE0FFF1FEF59FE4FB9
:10105000808191810E94290AF1E0FF1510F0F3943C
:1010600006C080917401826080937401FF240E9405
:101070005B09882321F00E946A090E943E070E94B2
:101080006C0D122F1519F1E0211708F0F0E0232F55
:101090002619E1E0321708F0E0E0B22FBF1B31E083
:1010A0002B1708F030E0E32B242F2719F1E042172B
:1010B00008F0F0E0A22FAE1B31E02A1708F030E074
:1010C000F32B252F281941E0521708F040E0E22FBA
:1010D000EF1B31E02E1708F030E0432B262F2919A3
:1010E00051E0621708F050E0622F641B31E02617D0
:1010F00008F030E0532B272F2A1941E0721708F02F
:1011000040E0322F351B532F31E0251708F030E037
:10111000432B282F2B1931E0821708F030E0822F63
:10112000841B482F81E0241708F080E0382B9C199D
:10113000931779F4442369F4552359F4662349F449
:10114000EE2339F4AA2329F4BB2319F4173908F440
:101150001FCF0E946002482E0E946C0D522E632EFB
:10116000742E852E962EA72EB82EC92E11CF1F9223
:101170000F920FB60F9211248F939F93EF93FF93CB
:10118000E0917701F09178018CB1E157FE4F8083B7
:1011900080917701909178014F9750F48091770179
:1011A000909178010196909378018093770104C023
:1011B0001092780110927701FF91EF919F918F919A
:1011C0000F900FBE0F901F9018951F920F920FB6A1
:1011D0000F9211242F933F938F939F93EF93FF933D
:1011E0002091790130917A0180917B0190917C016D
:1011F00028173907E9F0E0917901F0917A01E1557A
:10120000FE4F80818CB98091790190917A014F973E
:1012100050F48091790190917A01019690937A012E
:101220008093790109C010927A011092790104C06B
:1012300081E0809367015598FF91EF919F918F9185
:101240003F912F910F900FBE0F901F901895382F40
:10125000433078F5862F8550843058F5822F8150A1
:10126000823038F5442341F080B5806280BD423041
:1012700019F480B5806180BD223019F480B5886092
:1012800080BD653079F0663011F0683018F080B5B7
:10129000826080BD673030F080B5846080BD693089
:1012A00009F4529A90BD39B98AB188698AB980E047
:1012B000089581E008952091750130917601809123
:1012C00077019091780140E02817390709F041E053
:1012D000842F0895209175013091760180917701D6
:1012E000909178012817390711F420E022C0E0918D
:1012F0007501F0917601E157FE4F2081E091750173
:10130000F0917601E157FE4F108280917501909126
:1013100076014F9750F48091750190917601019676
:10132000909376018093750104C01092760110921B
:101330007501822F089580917B0190917C0120910D
:10134000790130917A0101968217930719F481E0AF
:1013500090E008958091790190917A01892B19F09C
:1013600080E090E0089580917B0190917C0120E0E5
:1013700030E04F9711F421E030E0C9010895482F83
:1013800080917B0190917C012091790130917A01CB
:10139000019682179307A1F38091790190917A01C8
:1013A000892B31F480917B0190917C014F9741F31F
:1013B000E0917B01F0917C01E155FE4F40838091EB
:1013C0007B0190917C014F9750F480917B0190912B
:1013D0007C01019690937C0180937B0104C0109264
:1013E0007C0110927B0180916701813021F4109281
:1013F0006701559A5D9A0895CF93DF93EC0103C07E
:1014000021960E94BF0988818823D1F7DF91CF916F
:1014100008951AB810BC10BC19B810927601109239
:10142000750110927A011092790110927801109250
:10143000770110927C0110927B0108952091810127
:10144000309182014091830150918401B901CA0118
:1014500008951F931FB7F89421E020937D01109207
:101460007E0110928001BC0140E050E019C08D91D6
:101470008095F90193E0EE0FFF1F9A95E1F7E40FD5
:10148000F51FE153FE4F80832F5F3F4F283031051A
:1014900071F74F5F5F4F685F7F4F4830510521F014
:1014A000DB0120E030E0E3CF1FBF1F910895682FDC
:1014B0007FB7F89481E080937D0110927E011092B5
:1014C000800120E030E060950FC0FA01E80FF91FBD
:1014D000E153FE4F6083019688309105B1F72F5F8D
:1014E0003F4F2830310549F080E090E0A901E3E06A
:1014F000440F551FEA95E1F7E8CF7FBF089580912B
:101500007E01869508958EB589608EBD82EC92EA43
:101510009BBD8ABD80E189BF80E00E94570A789414
:1015200040E050E091E01EC08FB7F894FB01E20F5D
:10153000F31FE153FE4FA081108290937D01109222
:101540007E01109280018FBF80917E018823E1F39C
:101550002F5F3F4F2830310539F74F5F5F4F4830DD
:10156000510549F020E030E0BA01F3E0660F771F43
:10157000FA95E1F7D9CFF894109281011092820187
:10158000109283011092840110927E0110928001CA
:10159000089589B78F7E89BF0895982F9C7F92BB4D
:1015A00098B3880F880F880F8871977E982B98BB07
:1015B0000895382F85B3837085BB88B3897F88BB36
:1015C000323058F025B381E090E002C0880F991FB7
:1015D0003A95E2F7282B25BB0EC048B3232F30E005
:1015E0002F5F3F4F81E090E002C0880F991F2A953E
:1015F000E2F7482B48BB6BBB000008951F920F9287
:101600000FB60F9211242F933F934F935F936F93D5
:101610007F938F939F93AF93BF93CF93DF93EF937A
:10162000FF938091800180917D01882321F01092A9
:101630007F0110927D0180E00E94CD0AC0E0D0E0E1
:10164000E0917F01F0E0A3E0EE0FFF1FAA95E1F724
:10165000EC0FFD1FE153FE4F60818C2F0E94D90AD1
:101660002196C830D10561F720917F0181E090E09B
:1016700002C0880F991F2A95E2F70E94CD0A809137
:101680007F01873030F480917F018F5F80937F01ED
:1016900007C010927F0180917E018F5F80937E0151
:1016A000109280018091810190918201A09183012B
:1016B000B09184010196A11DB11D80938101909389
:1016C0008201A0938301B0938401FF91EF91DF9198
:1016D000CF91BF91AF919F918F917F916F915F91CA
:1016E0004F913F912F910F900FBE0F901F90189523
:1016F00011B88CE080B90895982F84EA86BF06B6A9
:1017000007FEFDCF81B1887F883021F0803111F054
:1017100081E0089593B984E886BF06B607FEFDCF41
:1017200091B1987F983111F480E0089580E0903471
:1017300009F081E0089544EA34E824E946BF06B69A
:1017400007FEFDCF91B1987F983011F09031B1F73D
:1017500083B936BF06B607FEFDCF91B1987F9032B0
:1017600011F0983529F426BF06B604FCFDCFE6CF6C
:1017700008950E947C0B089584E986BF06B604FC98
:10178000FDCF089583B984E886BF06B607FEFDCF76
:1017900081B190E0887F883209F091E0892F089527
:1017A00084EC86BF06B607FEFDCF83B1089584E8BA
:1017B00086BF06B607FEFDCF83B10895BF92CF92D4
:1017C000DF92EF92FF920F931F93CF93DF937B01F2
:1017D0008C01D42EC52EB22E80E0E81680E0F806EB
:1017E00081E0080780E0180710F082EA01C080EA73
:1017F0000E947C0B882399F40E94C20B8E2D0E94BC
:10180000C20B8D2D9C2D9C01E90110E004C0899133
:101810000E94C20B1F5F1B15D0F30E94BC0BDF910F
:10182000CF911F910F91FF90EF90DF90CF90BF90DD
:101830000895DF92EF92FF920F931F937B018C012B
:10184000D42E80E0E81680E0F80681E0080780E00A
:10185000180710F082EA01C080EA0E947C0B8823FE
:1018600051F40E94C20B8E2D0E94C20B8D2D0E943E
:10187000C20B0E94BC0B1F910F91FF90EF90DF9065
:1018800008956F927F928F929F92AF92BF92CF9264
:10189000DF92FF920F931F93CF93DF934B015C0175
:1018A00080E0881680E0980681E0A80680E0B8060F
:1018B00018F092EAF92E02C080EAF82E642E7724FE
:1018C000C3010E94E00E8C016C01009769F18F2D1D
:1018D0000E947C0B882319F0CC24DD2425C080E0F5
:1018E0000E94C20B882D0E94C20B8F2D81600E9426
:1018F000B90BFF2453010894A108B10806C00E9447
:10190000D00BC00FD11F8883F394CF2DD0E0CA1520
:10191000DB05ACF30E94D70B060D171D01501040DC
:10192000F80180830E94BC0BC601DF91CF911F910B
:101930000F91FF90DF90CF90BF90AF909F908F90CE
:101940007F906F900895DF92EF92FF920F931F9315
:101950007B018C0180E0E81680E0F80681E0080752
:1019600080E0180718F032EAD32E02C020EAD22E07
:101970008D2D0E947C0B882311F010E00FC080E0B9
:101980000E94C20B8E2D0E94C20B8D2D81600E9481
:10199000B90B0E94D70B182F0E94BC0B812F1F91EF
:1019A0000F91FF90EF90DF900895CF93DF9383E442
:1019B0000E947C0B882319F020E030E011C0CFE0BA
:1019C000D2E00E94D00B899382E0C531D807C9F7D5
:1019D0000E94D70B88830E94BC0B9E01265030408A
:1019E000C901DF91CF91089583B78B6083BF8AEFE0
:1019F0008CBF89B7826089BF08951F920F920FB67E
:101A00000F9211241F932F933F934F935F936F93E4
:101A10007F938F939F93AF93BF93EF93FF938091A7
:101A20008601209187013091880140918901609160
:101A30008A01E0918B01A0918C0110918D01B82F4A
:101A4000BF5F91E0B81708F090E0F92FF20F81E046
:101A5000F21708F080E0782F730F81E0731708F019
:101A600080E0582F540F81E0541708F080E0382FA1
:101A7000360F81E0361708F080E0282F2E0F81E026
:101A80002E1708F080E0982F9A0F81E09A1708F03F
:101A900080E0810FB0938601F093870170938801F5
:101AA0005093890130938A0120938B0190938C018C
:101AB00080938D01FF91EF91BF91AF919F918F9195
:101AC0007F916F915F914F913F912F911F910F9057
:101AD0000FBE0F901F9018952091860130918701BD
:101AE000409188015091890160918A0170918B0128
:101AF00080918C0190918D0108958E3110F080E0DD
:101B00000895682F70E06E5F7F4F882777FD80957E
:101B1000982F0E94A30C08951F9360E070E080E06E
:101B200090E00E94A30C182F61E070E080E090E04C
:101B30000E94A30C412F50E0382F20E0422B532B62
:101B400087E0413E580710F040EE57E0CA011F9170
:101B50000895462F8E3150F4682F70E06E5F7F4FEE
:101B6000882777FD8095982F0E94190C08951F9360
:101B7000482F192F60E070E080E090E00E94190C7F
:101B800061E070E080E090E0412F0E94190C1F910D
:101B90000895EF92FF920F931F93EE24FF24870185
:101BA000C801B70140E00E94190C0894E11CF11C27
:101BB000011D111D80E0E81680E0F80682E00807AC
:101BC00080E0180769F71F910F91FF90EF9008953B
:101BD0000F931F93AB018C0126E0000F111F2A9574
:101BE000E1F7080F191F005E1F4F20E030E0C90128
:101BF000B80121E40E94DE0B1F910F9108959C0112
:101C000046E0220F331F4A95E1F7280F391F205E67
:101C10003F4F40E050E0CA01B90141E40E94410C4D
:101C200008958A3248F4E82FF0E0EE0FFF1FE55EDA
:101C3000FB4F6591749104C0EFE6F4E065917491F7
:101C400086E192E00E94E50F86E192E00895E7E0E8
:101C5000F0E0DF01A41BB109E21BF10923E0EE0F64
:101C6000FF1F2A95E1F7AE0FBF1FA80FB91F81E034
:101C700090E002C0880F991F6A95E2F72C91282BFB
:101C80002C930895E7E0F0E0DF01A41BB109E21B0B
:101C9000F10933E0EE0FFF1F3A95E1F7AE0FBF1FDA
:101CA000A80FB91F81E090E002C0880F991F6A95C4
:101CB000E2F780952C9128232C9308950E948D0F94
:101CC000089580E490E00E94E00E9C01009709F4E2
:101CD000FFCFFC01805C9F4F1192E817F907E1F7F5
:101CE000C90108950895BF92CF92DF92EF92FF92BB
:101CF0000F931F93CF93DF936C010E94610E7C01C1
:101D0000C0E0D0E0F601EC0FFD1F80816FE10E9482
:101D1000C00EB82E00E00CC0C7016C2F412F202F41
:101D20000E94270E1F5F1B15BCF30F5F083011F0D8
:101D300010E0F9CF2196C730D10521F7C7010E94E5
:101D4000290AC7010E945E0EDF91CF911F910F916A
:101D5000FF90EF90DF90CF90BF90089582E00895BC
:101D6000823050F4E82FF0E0EE0FFF1FE859FE4FED
:101D70000190F081E02D09950895A89508950895A2
:101D8000991B79E004C0991F961708F0961B881FCD
:101D90007A95C9F780950895AA1BBB1B51E107C02E
:101DA000AA1FBB1FA617B70710F0A61BB70B881FEB
:101DB000991F5A95A9F780959095BC01CD0108957A
:101DC000CF93DF93BC018230910510F462E070E0A4
:101DD000A0915402B0915502ED01E0E0F0E040E046
:101DE00050E021C0888199818617970769F48A811C
:101DF0009B81309719F09383828304C0909355029E
:101E000080935402FE0134C06817790738F44115F5
:101E1000510519F08417950708F4AC01FE018A8179
:101E20009B819C01E9012097E9F641155105A9F133
:101E3000CA01861B970B049708F4BA01E0E0F0E0B2
:101E40002AC08D919C91119784179507F9F4641716
:101E5000750781F412968D919C911397309719F024
:101E60009383828304C09093550280935402FD01B2
:101E700032964FC0CA01861B970BFD01E80FF91F70
:101E80006193719302978D939C9343C0FD0182816E
:101E900093819C01D9011097A1F6809152029091F3
:101EA0005302892B41F480916E0190916F019093C0
:101EB000530280935202409170015091710141157B
:101EC000510541F44DB75EB780916C0190916D0161
:101ED000481B590B209152023091530224173507A9
:101EE000B0F4CA01821B930B8617970780F0AB01F1
:101EF0004E5F5F4F8417950750F0420F531F50936A
:101F0000530240935202F9016193719302C0E0E0E1
:101F1000F0E0CF01DF91CF910895CF93DF93009749
:101F200009F450C0EC0122971B821A82A09154023E
:101F3000B0915502109709F140E050E0AC17BD0791
:101F400008F1BB83AA83FE0121913191E20FF31FB7
:101F5000AE17BF0779F48D919C911197280F391F07
:101F60002E5F3F4F3983288312968D919C91139752
:101F70009B838A834115510571F4D0935502C09318
:101F8000540220C012968D919C911397AD01009739
:101F900011F0DC01D3CFFA01D383C28321913191B7
:101FA000E20FF31FCE17DF0769F488819981280FAC
:101FB000391F2E5F3F4FFA01318320838A819B8135
:101FC00093838283DF91CF910895FB01DC0105901B
:0C1FD0000D920020E1F70895F894FFCF77
:101FDC0001FFFFFFFFFFFFFFFFFF818181818181F7
:101FEC00FFFF818181818181FFFF818181818181DD
:101FFC00FFFF818181818181FFFF818181818181CD
:10200C00FFFF818181818181FFFFFFFFFFFFFFFFC8
:10201C00FFFF010101FF8080FFFF010101FF8080B4
:10202C00FFFF010101FF8080FFFF010101FF8080A4
:10203C00FFFF010101FF8080FFFF010101FF808094
:10204C00FFFF010101FF8080FFFF010101FF808084
:10205C00FF7E818181FF8181817E818181FF8181F0
:10206C00817E818181FF8181817E818181FF81815E
:10207C00817E818181FF8181817E818181FF81814E
:10208C00817E818181FF8181817E818181FF81813E
:10209C00811E2222221E0202021E2222221E020265
:1020AC00021E2222221E0202021E2222221E0202D4
:1020BC00021E2222221E0202021E2222221E0202C4
:1020CC00021E2222221E0202021E2222221E0202B4
:1020DC0002A100E100210101BD0EBF0E200056023D
:0220EC000000F2
:00000001FF
